
 RASAPI16

 Start     Length     Name                   Class
 0001:0000 00CC3H     RASAPI16_TEXT          CODE
 0001:0CD0 0011DH     _TEXT                  CODE
 0001:0DED 00074H     INIT_TEXT              CODE
 0002:0000 00010H     NULL                   BEGDATA
 0002:0010 00096H     _DATA                  DATA
 0002:00A6 00000H     CDATA                  DATA
 0002:00A6 00000H     XIFB                   DATA
 0002:00A6 00000H     XIF                    DATA
 0002:00A6 00000H     XIFE                   DATA
 0002:00A6 00000H     XIB                    DATA
 0002:00A6 00000H     XI                     DATA
 0002:00A6 00000H     XIE                    DATA
 0002:00A6 00000H     XPB                    DATA
 0002:00A6 00000H     XP                     DATA
 0002:00A6 00000H     XPE                    DATA
 0002:00A6 00000H     XCB                    DATA
 0002:00A6 00000H     XC                     DATA
 0002:00A6 00000H     XCE                    DATA
 0002:00A6 00000H     XCFB                   DATA
 0002:00A6 00000H     XCF                    DATA
 0002:00A6 00000H     XCFE                   DATA
 0002:00A6 0000CH     DBDATA                 DATA
 0002:00B2 00000H     CONST                  CONST
 0002:00B2 00019H     HDR                    MSG
 0002:00CB 00082H     MSG                    MSG
 0002:014D 00002H     PAD                    MSG
 0002:014F 00001H     EPAD                   MSG
 0002:0150 00000H     _BSS                   BSS
 0002:0150 00000H     XOB                    BSS
 0002:0150 00000H     XO                     BSS
 0002:0150 00000H     XOE                    BSS

 Origin   Group
 0002:0   DGROUP

 Address   Export                  Alias

 0001:0000 LibMain                 LibMain
 0001:00C8 RasDial                 RasDial
 0001:02DE RasEnumConnections      RasEnumConnections
 0001:05FE RasEnumEntries          RasEnumEntries
 0001:091E RasGetConnectStatus     RasGetConnectStatus
 0001:0A84 RasGetErrorString       RasGetErrorString
 0001:0B0C RasHangUp               RasHangUp
 0001:008E WEP                     WEP

  Address         Publics by Name

 0000:0000  Imp  CALLPROC32W          (KERNEL.CALLPROC32W)
 0000:0000  Imp  FREELIBRARY32W       (KERNEL.FREELIBRARY32W)
 0000:0000  Imp  GETMODULEUSAGE       (KERNEL.48)
 0000:0000  Imp  GETPROCADDRESS32W    (KERNEL.GETPROCADDRESS32W)
 0000:0000  Imp  GETWINFLAGS          (KERNEL.132)
 0000:0000  Imp  GLOBALALLOC          (KERNEL.15)
 0000:0000  Imp  GLOBALFREE           (KERNEL.17)
 0000:0000  Imp  GLOBALLOCK           (KERNEL.18)
 0000:0000  Imp  GLOBALUNLOCK         (KERNEL.19)
 0000:0000  Imp  INITTASK             (KERNEL.91)
 0001:0E2F       LibEntry
 0001:0000       LibMain
 0000:0000  Imp  LOADLIBRARYEX32W     (KERNEL.LOADLIBRARYEX32W)
 0000:0000  Imp  LocalInit            (KERNEL.4)
 0000:0000  Imp  LSTRCPY              (KERNEL.88)
 0000:0000  Imp  OUTPUTDEBUGSTRING    (KERNEL.115)
 0000:0008  Abs  pAtomTable
 0000:0006  Abs  pLocalHeap
 0000:000E  Abs  pStackBot
 0000:000C  Abs  pStackMin
 0000:000A  Abs  pStackTop
 0001:00C8       RasDial
 0001:02DE       RasEnumConnections
 0001:05FE       RasEnumEntries
 0001:091E       RasGetConnectStatus
 0001:0A84       RasGetErrorString
 0001:0B0C       RasHangUp
 0000:0000  Imp  REGISTERWINDOWMESSAGE (USER.118)
 0002:0004       rsrvptrs
 0002:00A0       STKHQQ
 0001:008E       WEP
 0001:0B88       _AlignedAlloc
 0001:0C0C       _AlignedFree
 0002:0150       _edata
 0002:0150       _end
 0002:0010       _HRasApi32Dll
 0001:0C36       _MapErrorCode
 0002:0014       _UnRasDialEventMsg
 0000:9876  Abs  __acrtmsg
 0000:9876  Abs  __acrtused
 0000:9876  Abs  __acrtused2
 0000:D6D6  Abs  __aDBdoswp
 0002:00A2       __adbgmsg
 0002:00AA       __aDBrterr
 0001:0D50       __aFlmul
 0001:0D82       __aFlshl
 0001:0D8E       __aFuldiv
 0001:0D50       __aFulmul
 0002:00BA       __caption
 0002:0150       __edata
 0002:0150       __end
 0000:9876  Abs  __fptaskdata
 0001:0CE4       __NMSG_TEXT
 0001:0D1B       __NMSG_WRITE
 0001:0CE1       __wflags
 0000:0000  Imp  __WINFLAGS           (KERNEL.178)
 0002:00AC       ___aDBexit
 0002:00A8       ___aDBswpchk
 0002:00A6       ___aDBswpflg

  Address         Publics by Value

 0000:0000  Imp  LOADLIBRARYEX32W     (KERNEL.LOADLIBRARYEX32W)
 0000:0000  Imp  OUTPUTDEBUGSTRING    (KERNEL.115)
 0000:0000  Imp  GLOBALFREE           (KERNEL.17)
 0000:0000  Imp  REGISTERWINDOWMESSAGE (USER.118)
 0000:0000  Imp  INITTASK             (KERNEL.91)
 0000:0000  Imp  __WINFLAGS           (KERNEL.178)
 0000:0000  Imp  GETWINFLAGS          (KERNEL.132)
 0000:0000  Imp  GETMODULEUSAGE       (KERNEL.48)
 0000:0000  Imp  GLOBALALLOC          (KERNEL.15)
 0000:0000  Imp  GETPROCADDRESS32W    (KERNEL.GETPROCADDRESS32W)
 0000:0000  Imp  FREELIBRARY32W       (KERNEL.FREELIBRARY32W)
 0000:0000  Imp  GLOBALUNLOCK         (KERNEL.19)
 0000:0000  Imp  CALLPROC32W          (KERNEL.CALLPROC32W)
 0000:0000  Imp  LocalInit            (KERNEL.4)
 0000:0000  Imp  GLOBALLOCK           (KERNEL.18)
 0000:0000  Imp  LSTRCPY              (KERNEL.88)
 0000:0006  Abs  pLocalHeap
 0000:0008  Abs  pAtomTable
 0000:000A  Abs  pStackTop
 0000:000C  Abs  pStackMin
 0000:000E  Abs  pStackBot
 0000:9876  Abs  __fptaskdata
 0000:9876  Abs  __acrtused2
 0000:9876  Abs  __acrtmsg
 0000:9876  Abs  __acrtused
 0000:D6D6  Abs  __aDBdoswp
 0001:0000       LibMain
 0001:008E       WEP
 0001:00C8       RasDial
 0001:02DE       RasEnumConnections
 0001:05FE       RasEnumEntries
 0001:091E       RasGetConnectStatus
 0001:0A84       RasGetErrorString
 0001:0B0C       RasHangUp
 0001:0B88       _AlignedAlloc
 0001:0C0C       _AlignedFree
 0001:0C36       _MapErrorCode
 0001:0CE1       __wflags
 0001:0CE4       __NMSG_TEXT
 0001:0D1B       __NMSG_WRITE
 0001:0D50       __aFulmul
 0001:0D50       __aFlmul
 0001:0D82       __aFlshl
 0001:0D8E       __aFuldiv
 0001:0E2F       LibEntry
 0002:0004       rsrvptrs
 0002:0010       _HRasApi32Dll
 0002:0014       _UnRasDialEventMsg
 0002:00A0       STKHQQ
 0002:00A2       __adbgmsg
 0002:00A6       ___aDBswpflg
 0002:00A8       ___aDBswpchk
 0002:00AA       __aDBrterr
 0002:00AC       ___aDBexit
 0002:00BA       __caption
 0002:0150       __end
 0002:0150       _end
 0002:0150       __edata
 0002:0150       _edata

Program entry point at 0001:0e2f
